:100000000C9453010C9470010C9470010C947001C9
:100010000C9470010C9470010C9470010C9470019C
:100020000C9470010C942C090C9438080C94FF0863
:100030000C94A5080C94D2080C940B080C94780826
:100040000C94B8070C9470010C94C40E0C947001BD
:100050000C947A0E0C94BE010C9470010C947001F7
:100060000C9470010C9470010C9470010C9470014C
:100070000C9470010C9470010C94E90E0C947001B6
:100080000C949F0E0C94CA0A0C9470012F65727226
:100090006F722F6D73676C656E6774682F002F65C4
:1000A00072726F722F74797065746167322F002FCE
:1000B0006572726F722F74797065746167332F0087
:1000C0002F6572726F722F74797065746167342F47
:1000D000002F6572726F722F6D736773697A652F67
:1000E000002F6572726F722F636865636B73756D35
:1000F0000000000100080020004000800000010016
:10010000040000010008004000000100042F657297
:10011000726F722F444F522F002F6572726F722FC1
:100120005550452F002F6572726F722F46452F0074
:10013000303132333435363738394142434445461D
:10014000002F62746E31002F62746E32002F627461
:100150006E33002F62746E34002F62746E35002F80
:1001600062746E36002F62746E37002F62746E38C0
:10017000002F73777431002F736C6431002F6B6E16
:100180006231002F6164786C312F78002F616478C0
:100190006C312F79002F6164786C312F7A002F61D8
:1001A000646335002F61326432002F616463310073
:1001B0002F656E6331002F736C6432002F6B6E629B
:1001C00032002F736C6433002F6B6E6233002F7319
:1001D0006C6434002F6B6E6234002F6164633200F4
:1001E0002F61646333002F61646334002F6C656496
:1001F00031002F6C656432002F6C656433002F6C06
:10020000656434002F6C656435002F6C65643600BE
:100210002F736572766F31002F646973636F6E6E32
:10022000656374002F636F6E6E656374002F64697D
:1002300073636F6E6E656374002F636F6E6E6563BC
:1002400074002F696E32002F696E33002F696E348F
:10025000002F72657363616E002F786F6666002FE2
:100260006F757431002F6F757432002F6F75743392
:10027000002F6F757434002F7266696431002F721D
:1002800066696432002F7266696433002F72666992
:100290006434002F61646331002F61646332002F86
:1002A00061646333000011241FBECFEFD0E1DEBFD5
:1002B000CDBF11E0A0E0B1E0E6E4F0E300E00BBF69
:1002C00002C007900D92A230B107D9F715E0A2E065
:1002D000B1E001C01D92A93FB107E1F70C942016CF
:1002E0000C94000096B1987F982B96B9089527B189
:1002F0002F73992736E0880F991F3A95E1F7282B3D
:1003000027B90895379A359886E00E94720181E0F6
:100310000E9477013D98339A1092CC047894089506
:1003200033983798089597B1907E8F71982B97B92D
:100330000895349A369A089586B1992780749070FA
:1003400008951092CC0497B1907E8F71982B97B935
:10035000349A369A3699FECF84B1282F332785B147
:100360009927982F8827822B932B08950E94A1010B
:100370009695879596958795992708951F920F9240
:100380000FB60F9211248F938FEF8093CC048F912F
:100390000F900FBE0F901F9018950E94830C40E0A5
:1003A00052EC61E070E081E00E94470C08959927CB
:1003B00081309105A1F0823091051CF4892B21F048
:1003C00032C0029729F12FC081E00E94E20C6CE25A
:1003D0000E94710F81E00E94E20C69E62EC081E06C
:1003E0000E94E20C6CE20E94710F81E00E94E20C1C
:1003F00069E60E94710F81E00E94E20C69E60E94AA
:10040000710F81E00E94E20C60E00E94710F08957C
:1004100081E00E94E20C6CE20E94710F81E00E9478
:10042000E20C63E70AC081E00E94E20C6CE20E94E9
:10043000710F81E00E94E20C6EE40E94710F81E076
:100440000E94E20C60E0DBCF0F931F93CF93DF930A
:10045000EC0100E0FE012196149181E00E94E20C83
:10046000612F0E94710F0F5F1123A1F7802F992731
:1004700083709070892B69F081E00E94E20C60E04B
:100480000E94710F0F5F802F992783709070892BC6
:1004900099F7DF91CF911F910F9108951F93CF93FB
:1004A000DF93EC01162F81E00E94E20C6EEB0E94BC
:1004B000710F20E0FE018491882329F02F5FFE0157
:1004C000E20FF11DF8CF2F5F822F99278370907074
:1004D000892B11F02C7F2C5F120F81E00E94E20C1F
:1004E000612F0E94710FDF91CF911F9108950F939B
:1004F0001F93CF93DF93EC0100E0199181E00E94FC
:10050000E20C612F0E94710F0F5F1123B1F7802F52
:10051000992783709070892B69F081E00E94E20C2A
:1005200060E00E94710F0F5F802F99278370907099
:10053000892B99F7DF91CF911F910F9108950F9318
:100540001F93CF93DF9300E012E008C081E00E9488
:10055000E20CBE010E945F0F080F1F5FC12FDD2755
:1005600081E00E94E20CFC0184819581C817D907C3
:1005700068F381E00E94E20C602F0E94710FDF910E
:10058000CF911F910F9108950F931F93CF93DF93F6
:100590008C01EB0160E0FE018491882329F06F5FFC
:1005A000FE01E60FF11DF8CF6F5F862F992783704C
:1005B0009070892B11F06C7F6C5F6C5FC8010E949A
:1005C0004E02C8010E94240282E00E94D701CE019F
:1005D0000E9424020E949F0281E00E94980D809157
:1005E000EF048823E1F3DF91CF911F910F910895DC
:1005F0000F931F93CF93DF938C01EB0160E0888111
:10060000882331F06F5FFE01E60FF11D8081F8CF86
:100610006F5F862F992783709070892B11F06C7F04
:100620006C5F6C5FC8010E944E02C8010E942402E8
:1006300082E00E94D701CE010E9477020E949F02B1
:1006400081E00E94980D8091EF048823E1F3DF910F
:10065000CF911F910F910895EF92FF920F931F93E7
:10066000CF93DF93CDB7DEB728970FB6F894DEBFF0
:100670000FBECDBF7C0149835A836B837C830D837E
:100680001E832F8338876CE00E944E02C7010E94B0
:10069000240281E00E94D70181E00E94E20C6C817B
:1006A0000E94710F81E00E94E20C6B810E94710F29
:1006B00081E00E94E20CFE01319661810E94710F7F
:1006C00081E00E94E20C69810E94710F81E00E942A
:1006D000E20C68850E94710F81E00E94E20C6F813C
:1006E0000E94710F81E00E94E20C6E810E94710FE6
:1006F00081E00E94E20C6D810E94710F0E949F02B6
:1007000081E00E94980D8091EF048823E1F3289600
:100710000FB6F894DEBF0FBECDBFDF91CF911F9112
:100720000F91FF90EF9008950F931F93CF93DF9356
:10073000CDB7DEB724970FB6F894DEBF0FBECDBF9E
:100740008C0149835A836B837C8368E00E944E024C
:10075000C8010E94240280E00E94D70181E00E942B
:10076000E20C6C810E94710F81E00E94E20C6B81AF
:100770000E94710F81E00E94E20CFE0131966181BE
:100780000E94710F81E00E94E20C69810E94710F4A
:100790000E949F0281E00E94980D8091EF048823BF
:1007A000E1F324960FB6F894DEBF0FBECDBFDF9104
:1007B000CF911F910F9108950F931F938C0160E0CB
:1007C0000E944E02C8010E9424020E949F0281E002
:1007D0000E94980D8091EF048823E1F31F910F91FF
:1007E0000895109202011092DB041092D904109225
:1007F000E1041092E004109244011092430110921F
:10080000DA0440E450E063E071E08DEC94E00E9493
:100810000E0FE3E0F1E08FE31192815087FFFCCFF0
:100820000895909344018093430108950F931F937B
:10083000182F8091020199278830910509F4C9C0C9
:1008400089309105C4F48230910509F44BC083309E
:1008500091052CF4009751F1019769F1C2C18630DE
:10086000910509F444C1873091050CF0ACC105979E
:1008700009F455C1B6C18C30910509F450C08D30D2
:10088000910544F48A30910509F4E6C00B970CF009
:100890000BC1BBC08E30910509F46DC08E3091053F
:1008A0000CF44CC00F9709F47DC09BC11E3B09F0AE
:1008B0009AC181E031C11093DB041092D9041F3337
:1008C00010F482E029C1812F9927AA27BB278C0128
:1008D0009D014FE350E060E070E08CE890E00E9402
:1008E0002C0344C08091D904112349F0E82FFF273D
:1008F000ED5FFE4F10838F5F8093D90474C1E82FA2
:10090000FF27ED5FFE4F10838F5F8093D9049927F7
:1009100083709070892B09F066C18CE0FDC08091D6
:10092000D904E82FFF27ED5FFE4F10838F5F809380
:10093000D9041C3209F057C08DE0EEC08091D90473
:10094000E82FFF27ED5FFE4F10838F5F8093D90460
:10095000193611F48EE0E0C0812F9927AA27BB2712
:10096000AC01BD018EE990E00E94940381E00E94F9
:10097000650D87E0D1C08091D904E82FFF27ED5F96
:10098000FE4F10838F5F8093D904112311F48FE001
:10099000C3C0812F9927AA27BB27AC01BD018FEACD
:1009A00090E0E2CF8091D904E82FFF27ED5FFE4F62
:1009B00010838F5F8093D904112311F488E0ACC0B9
:1009C000812F9927AA27BB27AC01BD0180EC90E0BD
:1009D000CBCF8091D904E82FFF27ED5FFE4F108326
:1009E0008F5F8093D904812F9927AA27BB27B82F1F
:1009F000AA27992788278093DC049093DD04A0938D
:100A0000DE04B093DF0489E087C08091D904E82F29
:100A1000FF27ED5FFE4F10838F5F8093D904812FF6
:100A20009927AA27BB27AC01332722278091DC0412
:100A30009091DD04A091DE04B091DF04822B932B12
:100A4000A42BB52B8093DC049093DD04A093DE04EB
:100A5000B093DF048AE060C08091D904E82FFF27BB
:100A6000ED5FFE4F10838F5F8093D904812F99270C
:100A7000AA27BB272227382F492F5A2F8091DC0421
:100A80009091DD04A091DE04B091DF04822B932BC2
:100A9000A42BB52B8093DC049093DD04A093DE049B
:100AA000B093DF048BE038C08091D904E82FFF2792
:100AB000ED5FFE4F10838F5F8093D904212F332782
:100AC000442755278091DC049091DD04A091DE0439
:100AD000B091DF04822B932BA42BB52B8093DC04E5
:100AE0009093DD04A093DE04B093DF0414C08091E2
:100AF000D904E82FFF27ED5FFE4F1083E82FEF5F4B
:100B0000E093D9048091DB04E81709F06CC0FF275B
:100B1000ED5FFE4F108285E08093020164C08091FA
:100B2000D9044091DB04841781F09927AA27BB27B9
:100B30005527662777278C019D0181ED90E00E9463
:100B40002C0381E00E94650D4CC01092DA0490E005
:100B5000941750F4292FE3E0F1E08191280F9F5F73
:100B60009417D8F32093DA048091DA048117C1F442
:100B70008091430190914401892B99F18091DC048B
:100B80009091DD04A091DE04B091DF04E091430177
:100B9000F0914401AC01BD0183E091E0099521C0D1
:100BA00081E00E94650D8091DA049927AA27BB276E
:100BB000412F5527662777278C019D0181EE90E014
:100BC0000E942C030EC08091D9048F5F8093D904BA
:100BD000282F33278091DB0499270196281739079E
:100BE00011F4109202011F910F9108951F93182F75
:100BF00065E481E00E94EB0C612F81E00E94EB0C28
:100C0000812F0E9416041F910895039665E070E0FD
:100C10000E94D2179B0144275527DA01C90164E0DD
:100C2000880F991FAA1FBB1F6A95D1F7821B930BD0
:100C3000A40BB50B20E030E02817390718F42F5F1C
:100C40003F4FFACF0895883040F4E82FFF27EE0F8A
:100C5000FF1FEB5BFE4F11821082089593B7987FC0
:100C6000982B93BF08951092E2041092E30410921F
:100C7000E4041092E504089582E00E942E0612BE5C
:100C800087B7816087BF0E94330608959EB5987F1D
:100C9000982B9EBD089583E00E9446061DBC1CBC97
:100CA00087B7846087BF089595B5987F982B95BDC9
:100CB00008951092EA041092EB041092EC04109242
:100CC000ED04089584E00E94540614BC87B7806444
:100CD00087BF0E9459060895CF93C0E08C2F0E94D1
:100CE0002306CF5FC830D0F30E943C060E944B061B
:100CF0000E9462067894CF91089583B7E82FFF276A
:100D0000E770F070EE0FFF1FEF5FFE4F859194913B
:100D100008958EB5E82FFF27E770F070EE0FFF1FE4
:100D2000EF5FFE4F85919491089585B5E82FFF27D9
:100D3000E770F070EE0FFF1FEF50FF4F8591949119
:100D40000895883040F4E82FFF27EE0FFF1FEB5B7C
:100D5000FE4F718360830895DF92EF92FF920F93AD
:100D60001F93CF93DF93EC01D2B61092E60410925A
:100D7000E7041092E8041092E9040E947D069C01A9
:100D80004427552768EA7DEF80EE90E00E9408181E
:100D9000293B8DE8380786E0480780E05807C0F413
:100DA00087E2C131D807A0F4CE01AA27BB27BC0136
:100DB000CD010E94B317DC01CB01BC01CD0128EEAF
:100DC00033E040E050E00E94E617FA01E90111C06B
:100DD0007E0100271127CA01B90128EE33E040E067
:100DE00050E00E94E617C801B7010E94B317FC014A
:100DF000EB018091E6049091E704A091E804B091A2
:100E0000E9042227382F492F5A2F82B79927AA277A
:100E1000BB27282B392B4A2B5B2BCD0DD11DE11D78
:100E2000F11D2C173D074E075F0758F58091E6042A
:100E30009091E704A091E804B091E90485B7837E1E
:100E400085BF85B7806285BF889585B78F7D85BF53
:100E50008091E6049091E704A091E804B091E90440
:100E6000BA2FA92F982F882722B733274427552731
:100E7000822B932BA42BB52B8C179D07AE07BF0796
:100E8000A8F2DF91CF911F910F91FF90EF90DF902B
:100E900008958091E2049091E304A091E404B0915C
:100EA000E504BC01CD0108958091EA049091EB0422
:100EB000A091EC04B091ED04BC01CD0108958930FE
:100EC00031F48FB582608FBD8FB58E7F0AC08A30B6
:100ED00019F48FB5826002C08FB58D7F8FBD8FB53D
:100EE00081608FBD1BBC1ABC19BC18BC08959C0145
:100EF0008FB58E7F8FBD8FB582608FBD8EB58860B8
:100F00008EBD8EB580618EBD37BD26BD1BBC1ABCA3
:100F100019BC18BC08958FB58F778FBD8FB58F7BA7
:100F20008FBD08958FB58F7D8FBD8FB58F7E8FBD9F
:100F300008958FB58D7F8FBD8FB58E7F8FBD0E9439
:100F40008B070E94920708958FB580688FBD8FB57B
:100F50008F7B8FBD08958FB580628FBD8FB58F7EDB
:100F60008FBD08959BBD8ABD089599BD88BD089524
:100F70001F920F920FB60F9211242F933F934F930E
:100F80005F936F937F938F939F93AF93BF93EF93F1
:100F9000FF938091E2049091E304A091E404B09166
:100FA000E5040196A11DB11D8093E2049093E30432
:100FB000A093E404B093E5048091E6049091E704E3
:100FC000A091E804B091E9040196A11DB11D8093A0
:100FD000E6049093E704A093E804B093E9048091B9
:100FE000450190914601892B29F0E0914501F0914E
:100FF00046010995FF91EF91BF91AF919F918F911C
:101000007F916F915F914F913F912F910F900FBE04
:101010000F901F9018951F920F920FB60F921124E8
:101020002F933F934F935F936F937F938F939F93F0
:10103000AF93BF93EF93FF93809147019091480145
:10104000892B29F0E0914701F09148010995FF9122
:10105000EF91BF91AF919F918F917F916F915F9130
:101060004F913F912F910F900FBE0F901F901895A9
:101070001F920F920FB60F9211242F933F934F930D
:101080005F936F937F938F939F93AF93BF93EF93F0
:10109000FF938091EA049091EB04A091EC04B0914D
:1010A000ED040196A11DB11D8093EA049093EB0419
:1010B000A093EC04B093ED0480914F019091500106
:1010C000892B29F0E0914F01F09150010995FF9192
:1010D000EF91BF91AF919F918F917F916F915F91B0
:1010E0004F913F912F910F900FBE0F901F90189529
:1010F0001F920F920FB60F9211242F933F934F938D
:101100005F936F937F938F939F93AF93BF93EF936F
:10111000FF938091530190915401892B29F0E09124
:101120005301F09154010995FF91EF91BF91AF9157
:101130009F918F917F916F915F914F913F912F91EF
:101140000F900FBE0F901F9018951F920F920FB621
:101150000F9211242F933F934F935F936F937F933D
:101160008F939F93AF93BF93EF93FF938091490128
:1011700090914A01892B29F0E0914901F0914A01AF
:101180000995FF91EF91BF91AF919F918F917F91C1
:101190006F915F914F913F912F910F900FBE0F90E4
:1011A0001F9018951F920F920FB60F9211242F9334
:1011B0003F934F935F936F937F938F939F93AF93DF
:1011C000BF93EF93FF9380914B0190914C01892B3A
:1011D00029F0E0914B01F0914C010995FF91EF91BD
:1011E000BF91AF919F918F917F916F915F914F913F
:1011F0003F912F910F900FBE0F901F9018951F9247
:101200000F920FB60F9211242F933F934F935F933A
:101210006F937F938F939F93AF93BF93EF93FF93BE
:1012200080914D0190914E01892B29F0E0914D0163
:10123000F0914E010995FF91EF91BF91AF919F9170
:101240008F917F916F915F914F913F912F910F906F
:101250000FBE0F901F9018951F920F920FB60F920E
:1012600011242F933F934F935F936F937F938F93AB
:101270009F93AF93BF93EF93FF9380915101909110
:101280005201892B29F0E0915101F0915201099509
:10129000FF91EF91BF91AF919F918F917F916F914E
:1012A0005F914F913F912F910F900FBE0F901F9024
:1012B0001895809171008E7F8093710080917100EC
:1012C0008D7F8093710082E4809370000895109266
:1012D0009D0110929C0110929F0110929E0184E644
:1012E00090E00E945909809174008460809374009A
:1012F0001092560110925501809174008160809384
:1013000074008091740080648093740078940895D0
:1013100010929D0110929C0110929F0110929E01CB
:1013200084E690E00E94590985E4809374007894E3
:101330000895282F33272E7F30706111216020936C
:101340007200089590939D0180939C01089590935D
:101350009F0180939E010895809174008F70806A30
:10136000809374000895809174008F70806D8093D5
:1013700074000895809174008823E4F708958093A1
:101380007300809174008F7080688093740008955A
:10139000882329F0809174008F70806C04C0809144
:1013A00074008F708068809374000895809173003A
:1013B000992708958091710099270895282FDA01BF
:1013C0008091550190915601892BD1F782E090E0F0
:1013D00090935601809355012E7F2093570190E002
:1013E000961738F4E8E5F1E08D9181939F5F9617A9
:1013F000D8F31092780160937901809174008F7016
:10140000806A809374000895282FDA018091550135
:1014100090915601892BD1F783E090E0909356018B
:101420008093550121602093570110929A01609397
:101430009B01809174008F70806A8093740080910A
:10144000550190915601892BD1F790E0961738F409
:10145000EAE7F1E081918D939F5F9617D8F30895A5
:10146000282FFA0190E0809174008E7F80937400A1
:10147000809174008F70806A8093740080917400F2
:101480008823E4F72E7F20937300809174008F707F
:10149000806880937400809174008823E4F78091C1
:1014A0007100883189F4662381F081918093730003
:1014B000809174008F7080688093740080917400B4
:1014C0008823E4F76150EFCF91E0809174008F7032
:1014D000806D809374008091740084FFFCCF8091B4
:1014E0007400816080937400892F99270895282FB4
:1014F000DA0190E0809174008E7F80937400809177
:1015000074008F70806A80937400809174008823C7
:10151000E4F7216020937300809174008F708068DD
:1015200080937400809174008823E4F780917100A7
:10153000803409F5623088F0809174008F70806C7F
:1015400080937400809174008823E4F78091730085
:10155000FD01119680836150EDCF809174008F70F2
:10156000806880937400809174008823E4F78091F0
:1015700073008C9301C091E0809174008F70806D36
:101580008093740080917400816080937400892F2F
:10159000992708951F920F920FB60F9211242F933F
:1015A0003F934F935F936F937F938F939F93AF93EB
:1015B000BF93EF93FF9380919B0087FF03C081E06F
:1015C0000E94350E80917100887F282F33272036A6
:1015D000310509F4D0C0213631050CF041C0283264
:1015E000310509F489C029323105CCF420313105A7
:1015F00009F47FC0213131054CF42115310509F47E
:101600001FC12830310509F474C024C128313105C7
:1016100009F472C02032310509F48BC01BC120349B
:10162000310509F49CC0213431054CF420333105D7
:1016300009F47FC02833310509F480C00BC120357F
:10164000310509F480C0213531052CF428343105E9
:1016500009F46FC0FFC02835310509F45EC0FAC037
:101660002839310509F4DAC0293931050CF5283754
:10167000310509F480C0293731054CF4283631058D
:1016800009F479C02037310509F475C0E3C0283862
:10169000310509F4C3C0293831052CF4203831054F
:1016A00009F476C0D7C02039310509F471C0D2C021
:1016B000203B310509F48DC0213B31054CF4203A23
:1016C000310509F474C0283A310509F482C0C2C05A
:1016D000203C310509F4A9C0213C31052CF4283BFC
:1016E000310509F48AC0B6C0283C310509F49DC013
:1016F000B1C0809157010EC090917801809179011D
:101700009817B8F4E92FFF27E85AFE4F9F5F909390
:10171000780180818093730081C080919A01E82FC5
:10172000FF27E658FE4F9091730090838F5F809360
:101730009A01809174008F70806D7BC080917400DD
:101740008F70806876C080919A01E82FFF27E65855
:10175000FE4F9091730090838F5F80939A018091E8
:101760009A01282F332780919B01992701972817E9
:1017700039074CF053C085E090E090935601809378
:10178000550110929A01809174008F70806C4AC04C
:1017900080919A01E82FFF27E658FE4F9091730041
:1017A00090838F5F80939A01803268F337C0809175
:1017B00074008F70806C80937400E0919C01F091B4
:1017C0009D013097C1F16AE771E080919A01099516
:1017D00032C084E090E09093560180935501E091EF
:1017E0009E01F0919F01309731F068E571E080E251
:1017F0000995809379011092780190917801E92FF1
:10180000FF27E85AFE4F9F5F909378018081809375
:10181000730080917901981708F4B5CF8091740016
:101820008F7080688093740015C0809174008F70F1
:10183000806C8093740010925601109255010AC07A
:10184000809174008F70806D809374003093560186
:101850002093550180919B0087FF03C081E00E9487
:10186000350EFF91EF91BF91AF919F918F917F9135
:101870006F915F914F913F912F910F900FBE0F90FD
:101880001F901895809155019091560108951F93CE
:10189000182FDB01CA0173E0880F991FAA1FBB1F15
:1018A0007A95D1F79C01AD01220F331F441F551FBC
:1018B00088559240AF41BF4FBC01CD010E94E61751
:1018C000DA01C9010197112331F087E08093990073
:1018D0001092980005C089B9892F992780939000AC
:1018E0001F91089540E051E060EC72E088EF94E0D1
:1018F0000E940E0F40E051E060EC73E08AE095E05A
:101900000E940E0F08950E94720C1092C304109250
:10191000C20488ED80939A0040E855E260E070E0F0
:1019200081E00E94470C8FEF8093EF041092010535
:1019300010921505109214057894089540E051E036
:1019400060EA71E080EF94E00E940E0F40E250E008
:1019500060EA72E082E095E00E940E0F08950E9416
:101960009E0C1092C1041092C00488ED8AB940E820
:1019700055E260E070E080E00E94470C8FEF8093BA
:10198000EE0410920005109213051092120578943F
:1019900008950E94AF0C0E94830C0895823040F499
:1019A000E82FFF27EE0FFF1FE054FB4F718360838A
:1019B00008959927E3E0880F991FEA95E1F7805190
:1019C0009B4F08959927F3E0880F991FFA95E1F747
:1019D0008E5F9A4F0895982FE82FFF27DF01A251BD
:1019E000BB4F8C918823E9F3992319F060939C00F5
:1019F00001C06CB9E251FB4F10820895682F80E05E
:101A00000E94EB0C0895682F81E00E94EB0C089572
:101A1000CF93DF93EB01E82FFF27A3E0EE0FFF1F2B
:101A2000AA95E1F7E051FB4F82819381009751F035
:101A300084819581009731F0CF010E94180F88832F
:101A40008FEF90E0DF91CF910895CF93DF93CDB7E3
:101A5000DEB721970FB6F894DEBF0FBECDBFBE0133
:101A60006F5F7F4F81E00E94080D882319F0898104
:101A7000992702C08FEF9FEF21960FB6F894DEBF33
:101A80000FBECDBFDF91CF910895CF93DF93CDB738
:101A9000DEB721970FB6F894DEBF0FBECDBFBE01F3
:101AA0006F5F7F4F80E00E94080D882319F08981C5
:101AB000992702C08FEF9FEF21960FB6F894DEBFF3
:101AC0000FBECDBFDF91CF9108959927B3E0880F66
:101AD000991FBA95E1F780519B4F0E94A20F08957C
:101AE00020E030E0E82FFF2783E0EE0FFF1F8A950C
:101AF000E1F7E051FB4F84819581892B11F421E0BE
:101B000030E0C9010895992733E0880F991F3A956D
:101B1000E1F78E5F9A4F0E94710F0895682F80E061
:101B20000E94830D0895682F81E00E94830D08951F
:101B30001F93182F9927FC01E050FB4F2FEF2083B4
:101B400043E0880F991F4A95E1F78E5F9A4F0E94F4
:101B5000180F682F812F0E94EB0C1F910895AF92F0
:101B6000BF92CF92DF92EF92FF920F931F93CF938A
:101B7000DF93B82E8B01C82EDD24F60163E0EE0F53
:101B8000FF1F6A95E1F7EE5FFA4F84819581840F1C
:101B9000951F228133818217930760F54115510506
:101BA00049F1F801A1908F01C0E0D0E07A010894DA
:101BB000E108F108CE15DF0580F4F80121918F01CD
:101BC000C60153E0880F991F5A95E1F7622F8E5F87
:101BD0009A4F0E94710F2196EDCFEB2DFF27E05019
:101BE000FB4F8FEF80836A2D8B2D0E94EB0C8FEFC4
:101BF00090E002C080E090E0DF91CF911F910F91C3
:101C0000FF90EF90DF90CF90BF90AF900895CF936B
:101C1000DF93282FA82FBB27ED01C050DB4F888111
:101C20008823E1F0FD0173E0EE0FFF1F7A95E1F7E5
:101C3000EE5FFA4F84819581892B79F0222339F068
:101C40008AE095E00E94180F80939C000BC082E010
:101C500095E00E94180F8CB905C01882A251BB4FA5
:101C60008FEF8C93DF91CF910895CF93DF93C82F9F
:101C700080919B00992783FF03C08DE091E009C00C
:101C800082FF03C089E191E004C084FF04C085E2C3
:101C900091E00E94DC03CC2319F060919C0001C00C
:101CA0006CB12C2F3327E901C20FD31FFE01E05482
:101CB000FB4F80819181892B31F00190F081E02DE3
:101CC000862F099514C0E3E0220F331FEA95E1F750
:101CD000C90180519B4F0E94710F882341F4FE017E
:101CE000EE5EFA4F80819181019691838083DF912E
:101CF000CF9108951F920F920FB60F9211242F9338
:101D00003F934F935F936F937F938F939F93AF9383
:101D1000BF93EF93FF9380E00E94070EFF91EF9136
:101D2000BF91AF919F918F917F916F915F914F91F3
:101D30003F912F910F900FBE0F901F9018951F92FB
:101D40000F920FB60F9211242F933F934F935F93EF
:101D50006F937F938F939F93AF93BF93EF93FF9373
:101D600081E00E94070EFF91EF91BF91AF919F918B
:101D70008F917F916F915F914F913F912F910F9034
:101D80000FBE0F901F9018951F920F920FB60F92D3
:101D900011242F933F934F935F936F937F938F9370
:101DA0009F93AF93BF93EF93FF9380E00E94350E14
:101DB000FF91EF91BF91AF919F918F917F916F9123
:101DC0005F914F913F912F910F900FBE0F901F90F9
:101DD00018951F920F920FB60F9211242F933F93D5
:101DE0004F935F936F937F938F939F93AF93BF9323
:101DF000EF93FF9381E00E94350EFF91EF91BF9129
:101E0000AF919F918F917F916F915F914F913F9192
:101E10002F910F900FBE0F901F901895FC017183AA
:101E20006083538342831782168215821482089539
:101E3000CF93DF93EC01E0E02C813D81211531054A
:101E4000B9F08E819F81E881F981E80FF91FE08167
:101E500001969F838E836A817B818617970720F086
:101E60000E94D2179F838E83215030403D832C8364
:101E70008E2F9927DF91CF910895CF93DF93FC01A7
:101E8000EB012481358162177307A0F48681978165
:101E9000860F971F978386836281738186179707C2
:101EA00020F00E94D217978386832C1B3D0B35832D
:101EB000248302C015821482DF91CF910895FC0122
:101EC0008681978122813381860F971FB9010E94F5
:101ED000D2170190F081E02DE80FF91F808199273A
:101EE0000895CF93DF93EC01462F2C813D816A81C9
:101EF0007B812617370798F48E819F81820F931F6D
:101F00000E94D217E881F981E80FF91F40838C8184
:101F10009D8101969D838C838FEF90E002C080E0CD
:101F200090E0DF91CF910895FC0140E050E02481E2
:101F30003581828193812817390710F441E050E000
:101F4000CA010895FC011582148208959093C50476
:101F50008093C4040895E091C404F091C5040995E8
:101F60000895CF93DF93EC01892B61F0888188235A
:101F700049F0E091C404F091C504899109958881E4
:101F80008823B9F7DF91CF910895EF92FF920F93D5
:101F90001F93CF93DF938C017A01C0E0D0E0892BAF
:101FA00001F1CE0121968617970728F4F801819157
:101FB0008F018823B1F7C0E0D0E0CE15DF0588F4AB
:101FC000F8018081E091C404F091C504882319F0E0
:101FD0000F5F1F4F01C080E209952196CE15DF05E6
:101FE00078F3DF91CF911F910F91FF90EF900895BB
:101FF000CF93DF93EC01009779F0FC012196849157
:10200000882351F0E091C404F091C5040995FE01C4
:10201000219684918823B1F7DF91CF910895E091C3
:10202000C404F091C5048DE00995E091C404F091D9
:10203000C5048AE009950895E82FFF27EF70F07036
:10204000E05DFE4F8491E091C404F091C5040995D0
:1020500008951F93182F82958F700E941C10812F56
:102060000E941C101F9108950F931F938C01812FC4
:1020700099270E942910802F0E9429101F910F91EB
:102080000895EF92FF920F931F937B018C01C8017B
:10209000AA27BB270E943410C7010E9434101F9149
:1020A0000F91FF90EF9008952F923F924F925F9281
:1020B0006F927F928F929F92AF92BF92CF92DF9258
:1020C000EF92FF920F931F93CF93DF93CDB7DEB7BD
:1020D000A2970FB6F894DEBF0FBECDBF69A3242E22
:1020E0002AA337014801442351F017FF08C0EE240A
:1020F000FF248701E618F7080809190902C08401BE
:10210000730199A1692F772767FD70956150704021
:10211000222011F061507040362E18A22FE1422E7D
:10212000512C4C0E5D1EA82EBB24A7FCB094CB2CCA
:10213000DB2CC801B701A60195010E94E617DC015E
:10214000CB01FC01E05DFE4F84918F8FC801B70188
:10215000A60195010E94E61779018A013A94AFEF32
:102160003A1639F1C2010197E114F1040105110594
:10217000C1F02C01C801B701A60195010E94E61724
:10218000DC01CB01FC01E05DFE4F8491F201808314
:10219000C801B701A60195010E94E61779018A01DD
:1021A00004C02C01EAA1DC01EC933A94FFEF3F1646
:1021B000C9F62220B9F097FE05C08DE2D2018E93B8
:1021C0002D0110C0C2010197161417041804190438
:1021D0002CF42C018BE2F201808304C02C0180E2FC
:1021E000D2018C9339A03A94BFEF3B1661F0E09195
:1021F000C404F091C504D2018D912D0109953A9442
:10220000BFEF3B16A1F7A2960FB6F894DEBF0FBE44
:10221000CDBFDF91CF911F910F91FF90EF90DF9095
:10222000CF90BF90AF909F908F907F906F905F9076
:102230004F903F902F9008957F928F929F92AF92F0
:10224000BF92CF92DF92EF92FF920F931F93CF93A3
:10225000DF93CDB7DEB77888C988DA8863E1A62E28
:10226000B12CAC0EBD1E08C0882309F481C0E091DA
:10227000C404F091C504099596012F5F3F4F772064
:1022800021F0F6016901849103C0F60180816901A2
:10229000853251F72F5F3F4F772021F0F60169011A
:1022A000849103C0F60180816901282F332727FD1F
:1022B00030952436310591F02536310524F4233646
:1022C000310529F0D4CF2837310581F0D0CFF50181
:1022D00022E030E0A20EB31E8081C9CF5AE0852EE5
:1022E000912C40E1E42E47E2F42E04C030E1E32ECD
:1022F000F12C4701F50122E030E0A20EB31E00816F
:1023000011818436D9F417FF09C0109501951F4F2C
:10231000E091C404F091C5048DE2099532E0E31622
:10232000F10460F00E151F0548F4C7016AE070E083
:102330000E94D2177B0162307105A0F7C801B70176
:102340000E94D217FB01E05DFE4F8491E091C4042E
:10235000F091C5040995C801B7010E94D2178C01FC
:10236000C701B4010E94D2177B01672B39F784CFD4
:1023700080E090E0DF91CF911F910F91FF90EF905F
:10238000DF90CF90BF90AF909F908F907F900895F7
:10239000811188E0809316050895EF92FF921F93B4
:1023A000CF93DF93CDB7DEB721970FB6F894DEBF9A
:1023B0000FBECDBF182F80E8898380E00E94C8112E
:1023C000EE24FF24AE014F5F5F4F61E0812F0E943A
:1023D000300A882319F481E0E82EF12CC7012196F8
:1023E0000FB6F894DEBF0FBECDBFDF91CF911F9126
:1023F000FF90EF9008951F93CF93DF93CDB7DEB793
:1024000023970FB6F894DEBF0FBECDBF182F862FCF
:10241000807F90911605892B8983AE014F5F5F4FB6
:1024200061E0812F0E94300AAE014E5F5F4F62E093
:10243000812F0E94770A8A819927382F22278B8142
:102440009927822B932B23960FB6F894DEBF0FBEED
:10245000CDBFDF91CF911F910895962F97709295E0
:10246000907F692F0E94FB110895962F9695492F12
:102470005527262F332721703070220F331F220F4C
:10248000331F422B532B34E0440F551F3A95E1F78D
:10249000642F60680E94FB1108951092C804109286
:1024A000C7041092180510921705E9E1F5E089E0DC
:1024B0001192815087FFFCCF109223050E94AF0C30
:1024C00040E659E060E070E080E00E94470C129A1C
:1024D0001A980895282F8091180599278130910521
:1024E00089F0823091051CF4892B21F02BC00297D2
:1024F000C9F028C02A3041F581E080931805109278
:102500001705089580911705E82FFF27E75EFA4F1A
:1025100020838F5F809317058A30B0F082E080932C
:10252000180508952D3059F4E091C704F091C804BE
:10253000309729F069E175E08091C6040995109201
:1025400018050895109218050895CF93DF93CDB71D
:10255000DEB721970FB6F894DEBF0FBECDBFBE0128
:102560006F5F7F4F80E00E94080D882319F08981FA
:102570000E946A1221960FB6F894DEBF0FBECDBF3F
:10258000DF91CF9108959093C8048093C704089574
:1025900030E230932E0510922D053093300581E402
:1025A00091E0909332058093310582E28093340567
:1025B000109233053093360587E491E09093380507
:1025C0008093370584E280933A0510923905309361
:1025D0003C058DE491E090933E0580933D0586E2B5
:1025E0008093700510926F053093720583E591E03A
:1025F000909374058093730588E280937C05109214
:102600007B0530937E0589E591E09093800580936A
:102610007F058AE2809382051092810530938405BC
:102620008FE591E090938605809385058CE28093F9
:1026300088051092870530938A0585E691E090938E
:102640008C0580938B058EE280938E0510928D050C
:10265000309390058BE691E09093920580939105DD
:1026600084E38093400510923F053093420581E753
:1026700091E0909344058093430580E6809346055E
:10268000109245053093480587E791E090934A05FD
:102690008093490580E780934C0510924B05309359
:1026A0004E058DE791E09093500580934F0520E90A
:1026B00020935205109251052093540583E891E030
:1026C0009093560580935505209358051092570511
:1026D00040EA40935A058CE891E090935C05809322
:1026E0005B0520935E0510925D0580EC809360058C
:1026F00085E991E0909362058093610588E8809375
:10270000640510926305309366058EE991E090931D
:1027100068058093670583E980936A0510926905CF
:1027200010926C0584EA91E090936E0580936D059C
:1027300080E88093760510927505309378058AEAD3
:1027400091E090937A05809379054093A0051092CB
:102750009F053093A20580EB91E09093A4058093B0
:10276000A30582E680939405109293053093960515
:1027700086EB91E0909398058093970582E780938C
:102780009A051092990530939C058CEB91E09093FB
:102790009E0580939D0584E68093AC051092AB0561
:1027A0003093AE0582EC91E09093B0058093AF0535
:1027B00084E78093A6051092A5053093A80588ECC0
:1027C00091E09093AA058093A90586E68093B805C9
:1027D0001092B7053093BA058EEC91E09093BC054A
:1027E0008093BB0586E78093B2051092B1053093C4
:1027F000B40584ED91E09093B6058093B50582E829
:102800008093BE051092BD053093C0058AED91E01E
:102810009093C2058093C10584E88093C40510920B
:10282000C3053093C60580EE91E09093C805809370
:10283000C70586E88093CA051092C9053093CC0578
:1028400086EE91E09093CE058093CD0580E4809351
:10285000D0051092CF052FEF2093D2058CEE91E09A
:102860009093D4058093D30582E48093DC05109285
:10287000DB052093DE0582EF91E09093E0058093E5
:10288000DF0584E48093E2051092E1052093E405DE
:1028900088EF91E09093E6058093E50586E48093C8
:1028A000E8051092E7052093EA058EEF91E09093FA
:1028B000EC058093EB0588E48093EE051092ED051E
:1028C0002093F00584E092E09093F2058093F10567
:1028D0008AE48093F4051092F3052093F6058AE0CC
:1028E00092E09093F8058093F7058AE88093D605E7
:1028F0001092D5052093D80580E192E09093DA05F7
:102900008093D9050895C798C59AC79AC598089520
:10291000882319F0C798C59A0895C79AC59808954D
:102920008091C904982F93708F5F8093C904992375
:1029300019F481E08093CA040895CF93DF93CDB753
:10294000DEB721970FB6F894DEBF0FBECDBF698307
:102950009927FC01EE0FFF1FEE0FFF1FE80FF91F75
:10296000E80FF91FE153FA4FAE014F5F5F4F61E08F
:1029700081810E94DE0980E090E021960FB6F894F4
:10298000DEBF0FBECDBFDF91CF9108950F931F9390
:10299000CF93DF93CDB7DEB721970FB6F894DEBFA4
:1029A0000FBECDBF982F86E0989F90011124205D27
:1029B0003A4F892F99278C01000F111F000F111F0B
:1029C000080F191F080F191F035D1A4FA90161E0B5
:1029D000F80181810E94DE09AE014F5F5F4F61E027
:1029E000F80181810E94040A9981F8018281981777
:1029F00021F0928381E090E002C080E090E0219697
:102A00000FB6F894DEBF0FBECDBFDF91CF911F91FF
:102A10000F9108959927FC01EE0FFF1FEE0FFF1F86
:102A2000E80FF91FE80FF91FE35DFA4F828199273C
:102A3000AA27BB27AC01BD01848195810E94940324
:102A40000895BF92CF92DF92EF92FF920F931F9360
:102A5000CF93DF9300E010E06801F0E3EF2EF5E0A4
:102A6000FF2EEAE1BE2EE801CC0DDD1DC35DDA4F7D
:102A7000A70161E089810E94300A9881813051F478
:102A8000992331F06C817D8188E192E00E94C4023B
:102A900018820AC0992331F46C817D8184E292E02E
:102AA0000E94C40281E08883BA9486E090E0E80E38
:102AB000F91E0894C11CD11C0B5F1F4FB7FED3CF6A
:102AC00000E010E0680172EDE72E75E0F72E66E099
:102AD000B62EE801CC0DDD1DC153DA4FA70161E030
:102AE00089810E94300A9881813051F4992331F014
:102AF0006C817D818DE292E00E94C40218820AC03E
:102B0000992331F46C817D8189E392E00E94C402B3
:102B100081E08883BA9486E090E0E80EF91E08947C
:102B2000C11CD11C0B5F1F4FB7FED3CFDF91CF91DC
:102B30001F910F91FF90EF90DF90CF90BF9008957D
:102B40001F93CF93DF9313B3C12FDD279E01217015
:102B5000307080912405992781709070281739076B
:102B600039F0232B29F480E00E9483140E94211560
:102B70009E01247030708091240599278470907094
:102B800028173907A9F0CE019695879596958795D0
:102B900021E030E082279327AA27BB27817090701D
:102BA000A070B070AC01BD0182E492E00E94940379
:102BB0009E0120713070809124059927807190705A
:102BC00028173907B1F0CE01B4E096958795BA95EC
:102BD000E1F721E030E082279327AA27BB27817005
:102BE0009070A070B070AC01BD0187E492E00E94CB
:102BF00094039E012074307080912405992780747D
:102C0000907028173907B1F0A6E0D695C795AA9518
:102C1000E1F781E090E0C827D927CE01AA27BB279A
:102C200081709070A070B070AC01BD018CE492E036
:102C30000E94940310932405DF91CF911F91089572
:102C4000CEEFD0E1DEBFCDBF80EE87BB80EA88BB90
:102C50008AEA84BB85E585BB809324050E944B06E8
:102C60000E9467090E94CD010E94F10389E896E164
:102C70000E94110440E052EC61E070E081E00E94AB
:102C8000470C0E94C812DD24CD2C8D2D0E94831488
:102C90000E94211581E00E94460660E974E181E00E
:102CA0000E94A1068091CA04882341F11092CA04AF
:102CB0008C2D8170C3940E948814DD2400E010E004
:102CC0007801F801EE0DFF1DE35DFA4F8081882346
:102CD00041F08D2D0E94C614882319F08D2D0E947D
:102CE0000A15D3940894E11CF11C0B5F1F4F8AE175
:102CF0008D1538F703C089810E941604BE016F5FED
:102D00007F4F81E00E94080D8823A9F70E94A0153B
:102D1000C9CF8F929F92BF92CF92DF92EF92FF9294
:102D20000F931F93CF93DF93EC017A018B0161E541
:102D300072E00E94A917009719F59C015AE1B52E7F
:102D4000FC01E20FF31FE35DFA4F1082BA942F5F8C
:102D50003F4F0596B7FEF4CF80E090E09C0146E03F
:102D6000B42EFC01E20FF31FE153FA4F1082BA9424
:102D70002F5F3F4F0596B7FEF4CF0E94211582C00A
:102D800069E572E0CE010E94A917892B21F481E048
:102D90008093CA0477C06FE572E0CE010E94A91744
:102DA000892B71F481E090E0A0E0B0E0E822F92204
:102DB0000A231B23EF2811F0AF9864C0AF9A62C0BA
:102DC00065E672E0CE010E94A917892B71F481E0BB
:102DD00090E0A0E0B0E0E822F9220A231B23EF28CC
:102DE00011F0AD984FC0AD9A4DC06BE672E0CE01C8
:102DF0000E94A917892B71F481E090E0A0E0B0E077
:102E0000E822F9220A231B23EF2811F0AB983AC0DD
:102E1000AB9A38C061E772E0CE010E94A917892BF6
:102E200099F481E090E0A0E0B0E0E822F9220A23E2
:102E30001B23EF2811F0A99825C0A99A23C06E2D55
:102E40008B2D0E949D141EC0BB24CC24DD24460182
:102E5000F601E80DF91DE153FA4F8081882339F01E
:102E600064817581CE010E94A917892B41F3B39427
:102E70000894811C911CA5E0B0E0CA0EDB1EB6E0F0
:102E8000BB1530F7DF91CF911F910F91FF90EF901D
:102E9000DF90CF90BF909F908F90089599278130B9
:102EA000910579F0823091051CF4892B39F0089551
:102EB0008230910559F0039761F0089587E792E019
:102EC00002C08EE792E00E94F802089585E892E041
:102ED000FACF8CE892E0F7CF1F93182F0E94B6012B
:102EE000382F9927412F5527FA01EB5DFA4F2081A2
:102EF000821B9109892B59F1308343305105A1F090
:102F00004430510524F44130510529F020C04530AA
:102F1000510599F01CC0832F9927AA27BB27AC0124
:102F2000BD0183E992E011C0832F9927AA27BB270F
:102F3000AC01BD0189E992E008C0832F9927AA2737
:102F4000BB27AC01BD018FE992E00E9494031F9161
:102F50000895FB01DC018D910590801911F400208A
:102F6000D1F7990B0895629FD001739FF001829F62
:102F7000E00DF11D649FE00DF11D929FF00D839F08
:102F8000F00D749FF00D659FF00D9927729FB00DA5
:102F9000E11DF91F639FB00DE11DF91FBD01CF01B8
:102FA00011240895AA1BBB1B51E107C0AA1FBB1F18
:102FB000A617B70710F0A61BB70B881F991F5A95C5
:102FC000A9F780959095BC01CD010895A1E21A2E34
:102FD000AA1BBB1BFD010DC0AA1FBB1FEE1FFF1FBD
:102FE000A217B307E407F50720F0A21BB30BE40B0D
:102FF000F50B661F771F881F991F1A9469F7609554
:103000007095809590959B01AC01BD01CF0108950D
:1030100097FB092E05260ED057FD04D0D7DF0AD026
:10302000001C38F450954095309521953F4F4F4FF7
:103030005F4F0895F6F790958095709561957F4F55
:063040008F4F9F4F089521
:02304600010087
:00000001FF
